:020000040000FA
:10000000AF28A300360884008417340980058413C0
:10001000A3080319AA28F030A50022088038A400FC
:10002000F030A5030319A5000319A3030319AA2897
:100030002008A6002108A700163073202608A0007B
:100040002708A1004E20030120183408A21F3408FD
:10005000A20803190301A40F2F2880060D283028B9
:10006000000010280F39A0000310A00DA00D1F08DC
:10007000E039200401389F000030A10032307420A4
:100080009F149F1841281E08A10083161E08AA2845
:100090008001840AFF3E031D4828AA282108200465
:1000A0000319A00A8030201AA1062019A106A01861
:1000B000A106210DA00DA10DAA288316F8388105EF
:1000C0000F39810463000F308104AA28A301A20024
:1000D000FF30A207031CA307031CAA280330A100BA
:1000E000E33074206828A101F43EA000A109FE308D
:1000F000031C7D28A00703187A28A0076400A10F1D
:100100007A28000020188428201886280800A200D9
:1001100003309328A20001309328A20006309328D0
:10012000A20004309328A80023082102031D9A2866
:100130002208200204300318013003190230280578
:10014000031DFF30AA280038031DFF300405031DDE
:10015000FF30AA2883130313831264000800831658
:100160007E308F0090018312073099009501900135
:10017000831601309F00831283309F00203084005B
:1001800060304820A03084002030482083160D3095
:10019000850083128510831685108312051283163D
:1001A00005129630831266208514831685108312FB
:1001B0000130A300F4306720051683160512831260
:1001C0000130A300F4306720851083168510831258
:1001D00005128316051205308312B6002030B400D4
:1001E0007F30A2000A3001206400851DFC286400D5
:1001F000851DFB28F728EE296400051D0029D82954
:10020000640085108316851083120512831605126B
:10021000003083123220C2002108C3003230662031
:100220003E2107305D2007305D2007305D206400EF
:10023000051D1B291C2900290530B6002030B400FB
:100240007E30A200283001200230850683168510FA
:1002500083120130A3002C3067206400851D3D29E6
:100260006400851D3829051683160512831230296E
:10027000051283160512831200291C294208A000CA
:100280004308A1000330A30020309020BA004208A8
:10029000A0004308A1000230A300FD308A20BC006A
:1002A0003A0884003C08A320BC00BD0064003C0860
:1002B0003D0403196B2985148316851005308312BC
:1002C000B6002030B4007F30A2000A300120851033
:1002D0008316851083124208A0004308A100023053
:1002E000A300FD308720031D852985148316851002
:1002F00005308312B6002030B4007F30A2003C30BD
:10030000012085108316851083124208A00043083F
:10031000A1000330A30020308D20031D992905166C
:1003200083160512643083126620051283160512A7
:10033000831208004208A0004308A1000130A30076
:1003400090308720031DA8290512831605128312F9
:100350004208A0004308A1000130A30090308A2089
:10036000BA004208A0004308A1000230A3006C308C
:100370009020BC003A0884003C08A320BC00BD00CB
:1003800064003C083D040319C929051683160512AB
:1003900083124208A0004308A1000230A3006C3081
:1003A0008D20031DD72905168316051283120029F7
:1003B0006400051DED290230850683168510053081
:1003C0008312B6002030B4007F30A2001E3001201E
:1003D0000130A3002C306720D829002900303220BA
:1003E000C2002108C3000A3066204208A00043086A
:1003F000A1000330A3002A308D20031D032A051617
:100400008316051283124208A0004308A10003309E
:10041000A3002B308720031D112A85148316851015
:1004200083126400851D212A6400851D182A142A60
:100430000512831605128312851083168510831208
:08044000CA28112A6300222AD8
:02400E00D43F9D
:00000001FF
